:020000040000FA
:060000009EEF14F0120057
:0600080022EF00F01200DF
:06002A000200B0290000F5
:10003000F400000003000000802900000000000020
:04004000300000008C
:0C004400DACFE4FFE2CFDAFFE652E5522B
:10005000E5CFDAFF1100F26A9E6AA16A9D6AA06A82
:10006000F06A120000EF00F01200D9CFE6FFE1CFF6
:10007000D9FF020EE126010EDB6A010EDB50040AF5
:1000800001E1FDD0010A01E1F0D0060A01E1E2D070
:10009000010A25E0030A13E0010A01E0F9D0DF6A52
:1000A0000001A10EA86FDFCFA9F00001100EAA6F0A
:1000B000DE52010EDD6E086A01840196E9D015EC6E
:1000C00007F0640E085C05E1086ADE52050EDD6E7D
:1000D00005D001A603D0DE52020EDD6ED9D0DF506E
:1000E00024E1ABC030F0ACC031F0ADC032F0AEC0F6
:1000F00033F0AFC034F0B0C035F0B1C036F0B2C0AC
:1001000037F0B3C038F0B4C039F0B5C03AF0B6C07B
:100110003BF0B7C03CF0B8C03DF0B9C03EF0BAC04B
:100120003FF0DE52030EDD6E94D0100EDF5C24E152
:10013000ABC040F0ACC041F0ADC042F0AEC043F047
:10014000AFC044F0B0C045F0B1C046F0B2C047F017
:10015000B3C048F0B4C049F0B5C04AF0B6C04BF0E7
:10016000B7C04CF0B8C04DF0B9C052F0BAC053F0AF
:10017000DE52030EDD6E6DD0200EDF5C31E12F50BC
:1001800009E1ABC04EF0ACC04FF0ADC050F0AEC016
:1001900051F022D02F0409E1AFC04EF0B0C04FF0B3
:1001A000B1C050F0B2C051F017D0020E2F5C09E17F
:1001B000B3C04EF0B4C04FF0B5C050F0B6C051F06F
:1001C0000BD0030E2F5C08E1B7C04EF0B8C04FF063
:1001D000B9C050F0BAC051F0DE52030EDD6E39D016
:1001E000300EDF5C33E1040E2F5C09E1ABC04EF052
:1001F000ACC04FF0ADC050F0AEC051F023D0050EF2
:100200002F5C09E1AFC04EF0B0C04FF0B1C050F06C
:10021000B2C051F017D0060E2F5C09E1B3C04EF00A
:10022000B4C04FF0B5C050F0B6C051F00BD0070EBF
:100230002F5C08E1B7C04EF0B8C04FF0B9C050F025
:10024000BAC051F0DE52040EDD6E03D0DE52040E51
:10025000DD6E1ED0086A01840196100EDF26DFCF06
:10026000A9F0DE52010EDD6E13D01DD80196019467
:10027000010EE66E11EC08F0E5520BD009D00196A4
:100280000194020EE66E11EC08F0E55202D000D0A7
:10029000F4D6020EE15C02E2E16AE552E16EE5525B
:1002A000E7CFD9FF1200340E306E310E316E320EB0
:1002B000326E010E336E640E346E3F0E356E640E78
:1002C000366E3768B70E386E870E396E9C0E3A6EF2
:1002D000730E3B6ECE0E3C6E980E3D6E030E3E6E60
:1002E0003F6A406A320E416E030E426E3C0E436E10
:1002F000030E446E3C0E456E0A0E466E0A0E476EA5
:100300000A0E486E0A0E496E010E4A6E2C0E4B6E96
:10031000460E4C6EEC0E4D6E526A4B0E536E2F50C5
:1003200005E14E6A4F6A506A516A45D02F0407E1D1
:100330004E6A050E4F6E506A3C0E516E3CD0020E56
:100340002F5C06E14E6A050E4F6E5068516833D03F
:10035000030E2F5C07E14E6A3C0E4F6E506A3C0E56
:10036000516E29D0040E2F5C08E1030E4E6E840EF0
:100370004F6E506A3C0E516E1ED0050E2F5C07E189
:10038000030E4E6E840E4F6E5068516814D0060EE8
:100390002F5C08E1070E4E6E080E4F6E506A3C0E41
:1003A000516E09D0070E2F5C06E11C0E4E6E200E1A
:1003B0004F6E506851681200D9CFE6FFE1CFD9FFE8
:1003C000020EE126010EDB6A010EDB50090A01E193
:1003D00020D1030A01E116D1020A01E1FED00F0A81
:1003E00001E1EBD0010A13E0060A01E019D1DF6A4E
:1003F0000001A00EA86FDFCFA9F00001100EAA6FB8
:10040000DE52060EDD6E086A0184019609D1DF50C6
:1004100032E10001340EAB6F0001310EAC6F000110
:10042000320EAD6F0001010EAE6F0001640EAF6FB2
:1004300000013F0EB06F0001640EB16F0001B269A0
:100440000001B70EB36F0001870EB46F00019C0E60
:10045000B56F0001730EB66F0001CE0EB76F0001CD
:10046000980EB86F0001030EB96F0001BA6BDE522F
:10047000070EDD6EA1D0100EDF5C32E10001AB6B28
:100480000001320EAC6F0001030EAD6F00013C0E97
:10049000AE6F0001030EAF6F00013C0EB06F0001A4
:1004A0000A0EB16F00010A0EB26F00010A0EB36F9F
:1004B00000010A0EB46F0001010EB56F00012C0E91
:1004C000B66F0001460EB76F0001EC0EB86F000169
:1004D000B96B00014B0EBA6FDE52070EDD6E6CD0A9
:1004E000200EDF5C29E10001AB6B0001AC6B000169
:1004F000AD6B0001AE6B0001AF6B0001050EB06F7C
:100500000001B16B00013C0EB26F0001B36B000142
:10051000050EB46F0001B5690001B6690001B76B43
:1005200000013C0EB86F0001B96B00013C0EBA6FC0
:10053000DE52070EDD6E40D0300EDF5C2EE1000192
:10054000030EAB6F0001840EAC6F0001AD6B0001B8
:100550003C0EAE6F0001030EAF6F0001840EB06F52
:100560000001B1690001B2690001070EB36F00011B
:10057000080EB46F0001B56B00013C0EB66F0001B0
:100580001C0EB76F0001200EB86F0001B9690001A1
:10059000BA69DE52070EDD6E0FD0400EDF6EDF50FF
:1005A0000BE00001A9690001010EAA6F0001FD0E18
:1005B000AB6FDE52070EDD6E33D015EC07F0640E24
:1005C000085C05E1086ADE520A0EDD6E05D001A660
:1005D00003D0DE52080EDD6E23D0400EDF5C04E156
:1005E000DE52090EDD6E0DD0086A01840196100EF0
:1005F000DF260001A00EA86FDFCFA9F0DE52060EA5
:10060000DD6E0ED0040EE66E11EC08F0E55209D056
:1006100007D0050EE66E11EC08F0E55202D000D0CE
:10062000D3D6020EE15C02E2E16AE552E16EE552E8
:10063000E7CFD9FF1200D9CFE6FFE1CFD9FFE652CD
:100640008A9893888A988150100B01E0010EDF6E22
:100650009398DF5000D0E552E552E7CFD9FF120062
:100660008150400B01E0010E5B6E8150800B01E078
:10067000010EE8245A6E8250020B01E0010E040DB7
:10068000F3505A105B102F6E070ED8802F542F6E28
:10069000D2DF000907E090DE06DE8A9800019F9510
:1006A000FFD71FD00001A10EA86F0001A9690001AA
:1006B000010EAA6F086A01840196B7DB640E085C1C
:1006C00003E1F1DD0ED00CD001A60AD0FF0E00012F
:1006D000AB5D04E171DEE7DD04D002D0C6DC01D001
:1006E000ECD7120092809282928492869298929A8B
:1006F000CD0E936EFE0E946E8A6A929A899A0001CC
:100700009F9B928800019F9D949094908B900001F4
:100710009F9912003F0E9212EF0E936E949082906A
:100720009482948412000650020A18E0030A0EE034
:10073000010A01E04BD0070EC16E010EC26E3A0EE7
:10074000C06E9D9C010E066E076A40D00750040DD6
:10075000F3500109C26E020E066E38D0C282C2B2D8
:10076000FED70750090A29E00B0A20E0010A17E02A
:10077000020A0AE0010A01E026D0C4CF92F0C45078
:10078000546E010E076E1FD0C4CF93F0C450556E47
:1007900000B803D0030E076E01D0076A14D0C4CF8F
:1007A00094F0C450576E020E076E0DD0C4CF95F072
:1007B000C450566E090E076E06D0C4CF96F0C450D2
:1007C000586E076A00D0010E066E00D012008150EC
:1007D000400B01E0010E5D6E8150800B01E0010EC7
:1007E000E8245C6E8250020B01E0010E040DF3CF91
:1007F0005BF08150040B01E0010E080DF3CF5AF0BD
:100800008250040B01E0010E100DF3505A105B10E2
:100810005C105D1000019E6F02C097F003C098F05D
:1008200005C099F0F4C09AF004C09BF01200D9CF33
:10083000E6FFE1CFD9FFE652F26A54DF2BEC00F07D
:10084000D56AF29AB10ECD6ECF6ACE6A9D900E0E29
:10085000CA6ECC6AF90ECB6E9D92DF6A180EDF5C11
:1008600025E2DF50EA6A600FE96E000EEA22EF6AC5
:10087000DF50EA6A780FE96E000EEA22EF6ADF5075
:10088000EA6AA80FE96E000EEA22EF6ADF50EA6A10
:10089000900FE96E000EEA22EF6ADF50EA6AC00F9D
:1008A000E96E000EEA22EF68DF2AD8D7D9DE008889
:1008B000E552E552E7CFD9FF120000AA03D0009A13
:1008C00038EC13F0060E0001EA5D54E304010CBF9E
:1008D00009D000AC07D0009C6DB204D0010EE66ECA
:1008E000DDD8E5526D50020B11E10150010B0EE114
:1008F000180EE66E600EE66E000EE66E88EC12F0E4
:10090000E552E552E552000801E201806D50020B0C
:100910000CE1040104010C51800B07E101AA05D090
:10092000210EE66EBBD8E552019A6D50020B0CE128
:10093000040104010C51800B07E101A205D0320E25
:10094000E66EACD8E55201926D50020B11E1040144
:1009500004010C51800B0CE10150080B09E001A8C7
:1009600005D0310EE66E9AD8E552019801940196B1
:100970006DA200D001B03CD9120001A60DD0910E9D
:100980000001A85D09E10001A95106E1ABC02EF00C
:100990002EC09CF001960194120001B40AD000010F
:1009A000910EA86F0001A96B0001020EAA6F0196BB
:1009B000018412009EA203D09E92008001D000907C
:1009C00000A00CD00A50000808E20A060A5004E110
:1009D0000A0E0A6E008201D0009201D0009200A29D
:1009E0000CD00B50000808E20B060B5004E1640E1B
:1009F0000B6E008401D0009401D00094120000A07E
:100A000006D0205001E02006215001E0210600A27E
:100A100018D01350141005E01306000E145A059A4E
:100A200001D0058A1550161005E01506000E165A5D
:100A3000059C04D0938000019F81058C1F5001E02C
:100A40001F0600A42AD0A9DF0C5003E00C06059075
:100A500001D005800D5003E00D06059201D00582FE
:100A60000E5003E00E06059401D005840F501010BF
:100A700005E00F06000E105A059601D005861150AC
:100A800012100AE00001111C01E1121C03E0110622
:100A9000000E125A059801D005881200D9CFE6FF42
:100AA000E1CFD9FFE652DF6A180EDF5C09E2DF50C2
:100AB000EA6A780FE96E000EEA22EF6ADF2AF4D7BD
:100AC000FE0EDBCF78F0FE0EDB50110A01E18AD07A
:100AD000100A01E178D0330A50E0030A2AE0100A34
:100AE00001E081D00001160E796F020EDF6E180E44
:100AF000DF5C13E2DF50EA6A900FE96E000EEA2233
:100B0000EF50E66EDF50EA6A780FE96E000EEA22D7
:100B1000E552E750EF6EDF2AEAD7180EE66E780E40
:100B2000E66E000EE66E4CEC12F0E552E552E55230
:100B30005AD0010EDF6E180EDF5C13E2DF04EA6AA2
:100B4000A80FE96E000EEA22EF50E66EDF50EA6A67
:100B5000780FE96E000EEA22E552E750EF6EDF2AC9
:100B6000EAD7180EE66E780EE66E000EE66E4CECD6
:100B700012F0E552E552E55236D0F6C079F0020E99
:100B8000DF6E180EDF5C13E2DF50EA6AC00FE96E19
:100B9000000EEA22EF50E66EDF50EA6A780FE96E47
:100BA000000EEA22E552E750EF6EDF2AEAD7180E70
:100BB000E66E780EE66E000EE66E4CEC12F0E55234
:100BC000E552E55210D00001010E796F020EE66E7B
:100BD000780EE66E000EE66E4CEC12F0E552E55231
:100BE000E55201D000D0E552E552E7CFD9FF12001F
:100BF000D9CFE6FFE1CFD9FFE65260C0EFF00001A8
:100C0000F3050001F06F0001EF51910A32E0350A5F
:100C100006E0250A01E034D0018A019033D0040EA9
:100C20000001F05D24E301B422D061C0A8F062C0ED
:100C3000A9F063C0AAF0030EDF6E180EDF5C13E2AA
:100C4000DF28EA6A600FE96E000EEA22EF50E66ED6
:100C5000DF50EA6AA80FE96E000EEA22E552E7507B
:100C6000EF6EDF2AEAD701960188018400D0019057
:100C700009D0010E0001F05D01E30182019002D074
:100C8000019000D0E552E552E7CFD9FF1200948CD5
:100C9000948E8250400B03E08250800B02E1000EE4
:100CA00001D0010E00D01200050EE66EACEC14F07F
:100CB000E5521200948C948E8250400B03E08250D7
:100CC000800B02E1000E01D0010E00D01200ECDF1B
:100CD000829E949EE9DF829C949CE6DF000E00D009
:100CE0001200829E949E948CDFDF948E8250400B83
:100CF00003E08250800B02E1000E01D0010E00D013
:100D00001200D9CFE6FFE1CFD9FFFE0EDB5002E0A3
:100D1000948E02D0829E949EC7DF948CC5DF829C05
:100D2000949CC2DF000E00D0E552E7CFD9FF12003D
:100D3000D9CFE6FFE1CFD9FFE652948EB5DF948C90
:100D40008250800B01E0010EDF6EAEDF829C949C2E
:100D5000ABDFDF5000D0E552E552E7CFD9FF1200FC
:100D6000D9CFE6FFE1CFD9FFE652080EDF6EDF50A4
:100D70001DE0FE0EDBAE09D0010EE66EC2DFE552CD
:100D8000000902E0010E19D007D0E66ABADFE55289
:100D9000000902E0010E11D0FE0EDBCFF3FFF39E3F
:100DA000F346FE0EF3CFDBFFDF06E1D7C1DF00091C
:100DB00002E0010E02D0000E00D0E552E552E7CF6E
:100DC000D9FF1200D9CFE6FFE1CFD9FF020EE1260D
:100DD000080EDF6E010EDB6ADF5012E0010EDBCF82
:100DE000F3FFF39EF346010EF3CFDBFFA1DF000913
:100DF00003E0010EDB8002D0010EDB90DF06ECD7B2
:100E0000FE0EDBCFE6FF7DDFE552948E010EDB5058
:100E100000D05A6E020EE15C02E2E16AE552E16E38
:100E20005A50E552E7CFD9FF1200D9CFE6FFE1CF04
:100E3000D9FFE6520850640A01E1ECD0690A01E1E9
:100E4000E0D0010A01E1AED0060A01E19CD00C0A13
:100E500001E18CD0030A6DE0010A4AE0070A3CE098
:100E6000010A2BE0030A1EE0010A01E0D5D001507F
:100E7000040B08E00150080B05E1010E0001A81564
:100E800001080AE00150040B0CE00150080B09E1D5
:100E9000010E0001A81505E10DDF000902E0010EB9
:100EA000086EBAD08E0E5A6E0C0E5B6E5A505B10E6
:100EB00003E00DDF020E086EAFD0FE0E0001A81594
:100EC000E66E4EDFE552000903E1030E086E03D023
:100ED000F1DE010E086EA0D0A9C0E6FF41DFE552A9
:100EE000000903E1040E086E02D0640E086E94D06F
:100EF0000150040B0DE00150080B0AE1010E000146
:100F0000A815010805E1D6DEE2DE0A0E086E10D053
:100F10000150040B0BE00150080B08E1010E000129
:100F2000A81504E1096A050E086E02D0640E086E69
:100F300073D00001AA51095C16E2030E0924EA6A83
:100F4000A80FE96E000EEA22EFCFDFFFDFCFE6FF4A
:100F500007DFE552000904E1092A050E086E02D0F8
:100F6000640E086E02D0060E086E56D0BADE000976
:100F700007E0086A010E0001A8110001A86F02D065
:100F8000640E086E49D0010E0001A811E66EE8DE7D
:100F9000E552000904E1096A0C0E086E02D0640EE5
:100FA000086E3AD00001AA05095C12E2E66A0ADF7F
:100FB000E552E66E030E0924EA6AA80FE96E000EF8
:100FC000EA22E552E750EF6E092A0C0E086E18D09F
:100FD0000001AA05095C12E1010EE66EF3DEE5529E
:100FE000E66E030E0924EA6AA80FE96E000EEA22F3
:100FF000E552E750EF6E0D0E086E02D00D0E086E32
:101000000BD06FDE000903E0086A018602D0640E8F
:10101000086E02D066DE00D0E552E552E7CFD9FF78
:101020001200D9CFE6FFE1CFD9FFFE0EDB50040A54
:1010300024E0010A21E0070A1EE0030A1BE0020A7D
:1010400001E01CD00001F5510001F45D12E0000147
:10105000F62B180E0001F65D03E10001020EF66F9B
:101060000001F651EA6AC00FE96E000EEA22F4C0F0
:10107000EFFF04D003D002D001D000D0E552E7CF7B
:10108000D9FF12001B501C1004E01B06000E1C5A56
:1010900006D02AC01BF02BC01CF02950286E285007
:1010A0001CE01D501E1003E01D06000E1E5A1D50B0
:1010B0001E1012E12CC01DF02DC01EF000019FB5C6
:1010C00004D08A8800019F8507D0FF0E285C01E0CC
:1010D00028068A9800019F9503D08A9800019F9561
:1010E0001200D9CFE6FFE1CFD9FF030EE1262F5042
:1010F00009E1DE522C0EDD6E2C0EF36E020EF3CFE4
:10110000DBFF06D0010E31C0DBFF020E30C0DBFF7B
:101110005950545C06E2225002E0220601D00290AF
:1011200006D0320E225C02E2222A01D00280010E99
:10113000DB50555C0AE2265002E0260605D003A0EB
:1011400002D00382039403900ED0020EDB50555C54
:101150000AE33250265C02E2262A05D003B002D010
:1011600003840392038002920350010B01E0028288
:1011700000B873D03D50575C04E33C50D8805754BE
:1011800006E2235002E0230601D0029406D0230E8B
:10119000235C02E2232A01D002843B50565C04E324
:1011A0003A50D880565406E2245002E0240601D07A
:1011B000029606D0230E245C02E2242A01D0028685
:1011C0003950585C04E33850D880585406E2255012
:1011D00002E0250601D0029806D0230E255C02E22B
:1011E000252A01D002884C50E76E2E18E8AE02D0B6
:1011F000E73402D0E7502E5C02E3000E01D0010E6E
:10120000029EE8B0028E0A0E2E24DF6EDFCF5AF067
:101210004C50E76E5A18E8AE02D0E73402D0E750DF
:101220005A5C0BE24D50E76E2E18E8AE02D02E3419
:1012300003D0E750D8802E5402E3000E01D0010EF7
:10124000019EE8B0018EDFCFA3F001AE04D0000113
:10125000010EA46F02D00001A46B030EE15C02E258
:10126000E16AE552E16EE552E7CFD9FF120002B61E
:101270000AD04950196E1A6A4850176E186A0398B6
:10128000039A038621D081A410D04850176E186AA3
:1012900019501A1004E01906000E1A5A05D003B6A8
:1012A00002D0038A039803860FD04950196E1A6A38
:1012B0001750181004E01706000E185A05D003A6A0
:1012C00002D00388039A039612000250040B06E032
:1012D0000250080B03E00250100B02E1000E01D097
:1012E000010E029AE8B0028A0250400B06E002505A
:1012F000200B03E1038E039C08D00250400B05E154
:101300000250200B02E0038C039E029C0250200B33
:1013100001E0028C02AA04D0938200019F8304D0D2
:101320008A92939200019F93120000A82ED00098F9
:10133000FC0ED316D3A6FED772EC03F0085005E0DE
:10134000640E085C02E071DDF9D7086A0001900EB6
:10135000A86F0001010EA96F0001010EAA6F000124
:10136000AB6B018401960150080B05E1640E085C2B
:1013700002E05BDDF8D7086A019401960E0ECA6E92
:10138000CC6AF90ECB6E34EC13F01200008830EC0E
:1013900013F0085005E0640E085C02E046DDF9D762
:1013A000086A0001900EA86F0001010EA96F0001EC
:1013B000010EAA6F0001010EAB6F0184019601506E
:1013C000080B05E1640E085C02E02FDDF8D7086A1F
:1013D00001940196D382D3A6FED78AEC03F01200C3
:1013E0000001F4510001F55D06E00F0E0001F45D0F
:1013F00002E0F4C0F5F02F5005E103A002D0018C0B
:1014000001D0019C0001F451100A02E135EF0EF009
:101410001F0A01E1CED3010A01E1C3D3030A01E1AE
:1014200072D3010A01E114D31D0A01E103D31A0AA0
:1014300001E1A6D2010A01E142D2030A01E19AD1F7
:101440000E0A01E177D1010A01E15AD1030A01E153
:10145000ECD0160A01E1C2D0170A01E19FD0070AB9
:1014600001E189D0010A4DE0030A26E0010A02E009
:1014700047EF0EF08A9A00019F97938000019F81A9
:10148000929A899A00019F9B928800019F9D949057
:101490008B9000019F998A92939200019F938A9862
:1014A00000019F950001010EF46F2FC0A1F0000113
:1014B000130EA76F47EF0EF0FA0E2A6E2B6A020E7C
:1014C0002C6E2D6A020E296E1B6A1C6A1D6A1E6A2A
:1014D000226A236A246A256A266A026A056A036AFE
:1014E000046A03864850176E186A4950196E1A6AC2
:1014F000938000019F8101AC49DF0001020EF46F6F
:10150000C6D301BC03D03450596E02D0750E596E4B
:101510002F5006E00250010B03E00250020B0EE1D7
:101520002F5003E10150400B09E00150400B22E035
:10153000750E545C1FE3680E555C1CE3F6DE0394E5
:101540002F5004E10001040EF46F06D033500C6EEE
:1015500005900001030EF46F2F500CE04B0E2A6E25
:101560002B6A030E2C6E2D6A050E296E1B6A1C6AEF
:101570001D6A1E6A8CD302A00DD003A205D003926F
:101580000001100EF46F05D005A003D00001040E79
:10159000F46F03D00001100EF46F79D301AE77D34E
:1015A0000250010B06E12F5004E00001100EF46F11
:1015B00014D00350020B07E02F5005E00392000106
:1015C000100EF46F0AD0948000019F8902A605D006
:1015D00053501F6E0001130EF46F59D31F5024E1B6
:1015E0002F5003E1276A049203D04250276E0482F1
:1015F00043500E6E059441C015F040C016F0059C96
:1016000093908A9000019F91008A009C640E2A6E3C
:101610002B6A320E2C6E2D6A29681B6A1C6A1D6AA1
:101620001E6A0001050EF46F32D30250010B03E075
:101630000250080B06E12F5004E000010E0EF46F7B
:101640005ED00350020B07E02F5005E0039200012B
:101650000E0EF46F54D003B620D003B8039801AE39
:101660001BD001AC16D05550640804E23C0E0C6E41
:10167000059005D005A003D000010E0EF46F750E85
:10168000545C06E3680E555C03E30001060EF46F3C
:1016900003D00001060EF46F32D00550040B2FE08A
:1016A0000450020B2CE0275011E0270643500E6E29
:1016B00005940001DD0EA56F93908A9000019F9123
:1016C00041C015F040C016F0059C19D02F5017E00E
:1016D00051C011F050C012F005983650596E580E96
:1016E0002A6E020E2B6E320E2C6E2D6A030E296EA0
:1016F0001B6A1C6A1D6A1E6A00010D0EF46FC7D2B8
:101700008A9A00019F974BC013F04AC014F0059AC3
:10171000029C039E256A0298246A0296236A029418
:101720003550596E3E50206E3F50216E0001070E1D
:10173000F46FADD2205004E1929A898A00019F8B08
:10174000215004E19298899800019F8D205011E169
:1017500021500FE12F5004E03C0E0C6E059006D096
:1017600001AC04D03C0E0C6E059004900001090EF3
:10177000F46F8DD2286A8A8800019F850250010B80
:1017800017E12F5015E047500D6E059200010F0E26
:10179000F46F0A0E2A6E2B6A050E2C6E2D6A2968CC
:1017A0001B6A1C6A1D6A1E6A0001010EA06F81D0AF
:1017B00003AE1CD0039E2F5004E100010C0EF46F09
:1017C00011D047500D6E059200010F0EF46F0A0EF6
:1017D0002A6E2B6A050E2C6E2D6A29681B6A1C6AFC
:1017E0001D6A1E6A0001020EA06F63D002BE1BD0EC
:1017F0002F5004E100010C0EF46F11D047500D6E14
:10180000059200010F0EF46F0A0E2A6E2B6A050E68
:101810002C6E2D6A29681B6A1C6A1D6A1E6A0001EB
:10182000030EA06F46D00350020B1DE02F501BE0AB
:101830000550010B18E003924FC00FF04EC010F09E
:10184000059600010A0EF46FC80E2A6E2B6A640E0C
:101850002C6E2D6A29681B6A1C6A1D6A1E6A0001AB
:10186000040EA06F26D003AA08D0039A00010C0E24
:10187000F46F0001050EA06F1CD001AC1AD05550BA
:10188000640804E23C0E0C6E059013D005A011D044
:1018900093908A9000019F91008C009A41C015F0AE
:1018A00040C016F0059C3C0E0C6E05900001110E18
:1018B000F46F05AA03D08A8A00019F87E8D102B09D
:1018C00012D047500D6E059200010F0EF46F0A0EF4
:1018D0002A6E2B6A050E2C6E2D6A29681B6A1C6AFB
:1018E0001D6A1E6A4CD003AE13D0039E47500D6E86
:1018F000059200010F0EF46F0A0E2A6E2B6A050E78
:101900002C6E2D6A29681B6A1C6A1D6A1E6A37D0F4
:1019100002BE12D047500D6E059200010F0EF46FFB
:101920000A0E2A6E2B6A050E2C6E2D6A29681B6A18
:101930001C6A1D6A1E6A23D003A405D0039400010B
:10194000090EF46F1CD003AA05D0039A00010C0EF7
:10195000F46F15D005A613D093908A9000019F9143
:10196000008C009A41C015F040C016F0059C45500F
:101970000E6E05944450276E00010B0EF46F87D154
:1019800002B012D047500D6E059200010F0EF46F99
:101990000A0E2A6E2B6A050E2C6E2D6A29681B6AA8
:1019A0001C6A1D6A1E6A45D003AE13D0039E4750C1
:1019B0000D6E059200010F0EF46F0A0E2A6E2B6A4F
:1019C000050E2C6E2D6A29681B6A1C6A1D6A1E6A28
:1019D00030D002BE12D047500D6E059200010F0E9E
:1019E000F46F0A0E2A6E2B6A050E2C6E2D6A29687A
:1019F0001B6A1C6A1D6A1E6A1CD003AA05D0039AC2
:101A000000010C0EF46F15D005A413D027500EE082
:101A1000270645500E6E059441C015F040C016F0E3
:101A2000059C93908A9000019F9103D000010C0EB9
:101A3000F46F2DD105A005D0048000010C0EF46FC9
:101A400006D003AA04D0039A00010C0EF46F1FD134
:101A50008A9A00019F97929A899A00019F9B928887
:101A600000019F9D4850176E186A4950196E1A6AF6
:101A70002F501DE10150400B0BE00350080B08E113
:101A80000480010E000904E000010E0EF46F0ED078
:101A9000640E2A6E2B6A320E2C6E2D6A29681B6A20
:101AA0001C6A1D6A1E6A0001050EF46F2BD002A28B
:101AB00012D004923450596E640E2A6E2B6A320E84
:101AC0002C6E2D6A29681B6A1C6A1D6A1E6A000139
:101AD000050EF46F17D051C011F050C012F00598E8
:101AE0003650596E580E2A6E020E2B6E320E2C6E28
:101AF0002D6A030E296E1B6A1C6A1D6A1E6A00018C
:101B00000D0EF46FC4D00250010B14E12F5012E0FF
:101B100046500D6E059200010F0EF46F0A0E2A6EEC
:101B20002B6A050E2C6E2D6A29681B6A1C6A1D6AB9
:101B30001E6A36D00250800B14E12F5012E046503E
:101B40000D6E059200010F0EF46F0A0E2A6E2B6ABD
:101B5000050E2C6E2D6A29681B6A1C6A1D6A1E6A96
:101B60001FD02F5015E00350040B12E03450596E73
:101B70000001020EF46F4B0E2A6E2B6A030E2C6EC0
:101B80002D6A050E296E1B6A1C6A1D6A1E6A08D022
:101B90000550100B05E02F5003E000010E0EF46F0E
:101BA00076D094908B9000019F990001100EF46FF5
:101BB0006ED00550020B02E152500FE0929A899AC2
:101BC00000019F9B928800019F9D94908B90000143
:101BD0009F990001100EF46F47D0090E0001F55DCA
:101BE0000DE10250010B09E00250200B06E002500B
:101BF000800B03E00001090EF46F36D00A0E0001DD
:101C0000F55D18E10250010B14E00250200B11E0C9
:101C10000250800B0EE0C80E2A6E2B6A640E2C6EEA
:101C20002D6A29681B6A1C6A1D6A1E6A00010A0E59
:101C3000F46F1AD00D0E0001F55D16E10250010B94
:101C400013E00250800B10E0580E2A6E020E2B6E2D
:101C5000320E2C6E2D6A030E296E1B6A1C6A1D6AD9
:101C60001E6A00010D0EF46F12D0FA0E2A6E2B6A56
:101C7000020E2C6E2D6A020E296E1B6A1C6A1D6AEA
:101C80001E6AC6EC09F00001020EF46F00D00F0EC0
:101C90000001F45D05E0030EE66E11EC08F0E5527C
:101CA000120000B80ED097EC14F0DAEC04F0FFEC60
:101CB00004F0E7EC03F015EC07F0BDEC04F05DEC8C
:101CC00004F093EC03F000A805D071EC08F042ECAE
:101CD00008F00ED000A20CD071EC08F000B802D0D1
:101CE00037EC09F0090E0001F45D02E042EC08F067
:101CF00000B802D065EC09F0F0EC09F0F5C0A6F0F0
:021D00001200CF
:0E1D02006C5002E0000E01D0010E00090BE053
:101D1000040100513C0BE842E8420D0802E10CD8F6
:101D200001D042D808D06C5002E0000E01D0010E64
:101D3000040901E04BD81200D9CFE6FFE1CFD9FF6B
:101D4000E6520001E26B0001E36B0001E86BE96B16
:101D50001EEC10F0DF6ADF505A6E5B6A010E5A5CAF
:101D6000000E5B581BE20001E35101E017D0F76A57
:101D7000DF34FE0BF736F66E6D0EF626280EF722D0
:101D80000900F5CF5AF00800F5CF5BF004D05BC036
:101D9000FAFF5A50F96EFBDFDF2ADDD7F0D8E552A3
:101DA000E552E7CFD9FF1200020E0001E25D0CE11F
:101DB000A4D8040100BD04D00401C80E006F03D0F4
:101DC0000401880E006F01D029D91200040E000111
:101DD000EA5D0CE112C46EFF6E50000804E20001DF
:101DE000050EEA6F03D00001030EEA6F0001E20561
:101DF0000CE10DD8040104BD04D00401C80E046F29
:101E000003D00401880E046F01D008D91200D9CF85
:101E1000E6FFE1CFD9FF020EE1260001080EE85DE2
:101E2000000EE95905E2E8C0DEFFE9C0DDFF03D09E
:101E3000080EDE6EDD6A0401049304010491010EB4
:101E4000DB5004010413DFCF05F4000EDB5000016A
:101E5000E85F010EDB500001E95B0001180EE66F40
:101E6000040EE76F0001EBA320D0D9CFE9FFDACF52
:101E7000EAFFEE50ED1018E0E4C0F6FFE5C0F7FF12
:101E80000800F550E6C0E9FFE7C0EAFFEF6E000189
:101E9000E62B000EE7230001E42B000EE523DF060E
:101EA000010E01E2DB06E1D71ED0D9CFE9FFDACF80
:101EB000EAFFEE50ED1017E0E4C0E9FFE5C0EAFFED
:101EC000EF50E6C0E9FFE7C0EAFFEF6E0001E62B46
:101ED000000EE7230001E42B000EE523DF06010ED0
:101EE00001E2DB06E2D7020EE15C02E2E16AE552C2
:101EF000E16EE552E7CFD9FF1200D9CFE6FFE1CF7F
:101F0000D9FF020EE126030E04010015E76E010E53
:101F1000E7CFDBFF01C4DFFFDE500001E827DD5023
:101F20000001E9230001180EE46F040EE56FD9CF1C
:101F3000E9FFDACFEAFFEE50ED1017E0E4C0E9FF69
:101F4000E5C0EAFFEF50E6C0E9FFE7C0EAFFEF6E49
:101F50000001E62B000EE7230001E42B000EE52331
:101F6000DF06010E01E2DB06E2D7020EE15C02E2CF
:101F7000E16AE552E16EE552E7CFD9FF12000001B8
:101F8000E3510FE10401080E016F0401100E026F0E
:101F9000040E036F0401840E006F0401840E046FAD
:101FA0003BD0040110AF25D00001E8510401165DBB
:101FB0000001E9510401175904E216C4E8F017C4FE
:101FC000E9F025DF0001010EE26F0401080E016F48
:101FD0000401100E026F040E036F0401800E006FE7
:101FE0000401180E066F040E076F0401C80E046F7B
:101FF00013D00001020EE26F0401056B0401C80E4C
:10200000046F0401080E016F0401180E026F040E24
:10201000036F0401C80E006F6D9812000001E26B9F
:102020000401080E016F0401100E026F040E036F0D
:0C2030000401880E006F0401046B120014
:04203C00040110513A
:10204000600BE842E842E842E842E842000901E069
:1020500058D004011151070A53E00B0A51E0070A56
:1020600042E0010A2CE00B0A28E0020A26E0030AFB
:1020700022E0080A12E0010A0EE00F0A0AE0030A51
:1020800001E03ED00001010EE36F0001040EEA6F93
:1020900038D038D836D093D834D00001010EE36F51
:1020A0000001EC0EE46F000EE56F0001EB93000100
:1020B000010EE86F26D0ABD824D0FAD822D0000188
:1020C000010EE36F040114510001E46FE56BED0EA6
:1020D0000001E427000E0001E5230001EB9300015D
:1020E000010EE86F0ED00001010EE36F04011451E0
:1020F000EA6AED0FE96E000EEA2212C4EFFF01D08A
:1021000000D01200800E0401105D58E1040113514B
:10211000030A34E0010A10E0030A01E04DD0000197
:10212000010EE36F00011C0EE46F270EE56F120E27
:102130000001E86FE96B40D00001010EE36F04017C
:102140001251F66EF76AD890F636F736610EF6261B
:10215000280EF7220900F5CFE4F00A00F5CFE5F0EC
:10216000020E0001F76AE425F66EE551F722090038
:10217000F5CFE8F00A00F5CFE9F01ED00001010E1E
:10218000E36F04011251F66EF76AD890F636F7360F
:10219000650EF626280EF7220900F5CFE4F00A00B6
:1021A000F5CFE5F0E4C0F6FFE5C0F7FF0800F55015
:1021B0000001E86FE96B00D00001EB831200000121
:1021C000010EE36F0F0EE66E710EE66E0F0EE66EF9
:1021D00079EC13F0E552E552E552010EE66EED0E94
:1021E000E66E000EE66E79EC13F0E552E552E5522C
:1021F00012C4ECF00401125104E10001050EEA6F73
:1022000005D00001060EEA6F34EC12F01200040152
:10221000186B0401196B040110511F0B020A15E021
:10222000030A0FE0010A01E035D00001010EE36F5F
:1022300002D0040118810001EBA102D0040118832F
:1022400029D00001010EE36F25D00001010EE36FDC
:10225000040114510F0B080DF3505B6A000F5A6E06
:10226000040E5B2204011451800B01E0010E040DE9
:10227000F35000015A24E66F000E5B20E76FE6C0C2
:10228000E9FFE7C0EAFFEF50040B03E00401010E91
:10229000186F00D00001E3050AE10001180EE46F99
:1022A000040EE56F0001EB930001020EE86F1200CF
:1022B0000401120511E1040110511F0B00090CE18A
:1022C0000001010EE36F030E0401115D03E1000143
:1022D000EB8102D00001EB91040112513EE10401B7
:1022E00010511F0B020839E1040114510F0B0009B2
:1022F00034E00001010EE36F040114510F0B080DCF
:10230000F3505B6A000F5A6E040E5B2204011451F5
:10231000800B01E0010E040DF35000015A24E66F1A
:10232000000E5B20E76F030E0401115D07E1840ED0
:10233000E6C0E9FFE7C0EAFFEF6E0FD0040114AF7B
:1023400006D0E6C0E9FFE7C0EAFFEF6A06D0880ED4
:0C235000E6C0E9FFE7C0EAFFEF6E1200F4
:04235C000401105117
:102360001F0B010801E07DD00401145101E079D078
:10237000060E0401115D2FE104011351230A28E028
:10238000010A13E0030A01E024D00001020EE36F0A
:102390000001EC0505E10001400EE46F270EE56F3A
:1023A000090E0001E86FE96B14D00001020EE36F23
:1023B0000001EC0505E10001990EE46F270EE56FC1
:1023C0000001EC0504E1C80E0001E86FE96B01D0E3
:1023D00000D00001EB8304011051600BE842E84299
:1023E000E842E842E842010801E03BD00401115113
:1023F0000B0A31E0080A21E0090A19E0080A09E09D
:102400000B0A05E0080A01E02CD02CD82AD02BD8E2
:1024100028D00001020EE36F0001F10EE46F000E00
:10242000E56F0001EB930001010EE86F1AD0000187
:10243000020EE36F13C4F1F014D00001020EE36F3B
:102440000001F20EE46F000EE56F0001EB93000156
:10245000010EE86F06D00001020EE36F12C4F2F025
:1024600000D01200120012000001F36B1E0E716EFC
:102470000401180E096F0401200E0A6F040E0B6F81
:102480000401880E086F0401380E0E6F040E0F6FE2
:102490000401400E0C6F1200D9CFE6FFE1CFD9FF47
:1024A000E652FC0EDB50180805E2180EF36EFC0E27
:1024B000F3CFDBFFDF6AFC0EDB50DF5C19E2DF509D
:1024C000E76EFD0EDBCFE9FFFE0EDBCFEAFFE75044
:1024D000E926000EEA22EF50E66EDF50EA6A380F76
:1024E000E96E040EEA22E552E750EF6EDF2AE3D7E9
:1024F000FC0EDBCF0DF4400E04010C1704010C7D23
:10250000880E04010C13E552E552E7CFD9FF120003
:10251000D9CFE6FFE1CFD9FF0001F36B040108BF7B
:1025200039D0FC0EDBCF5AF004010951D8805A543F
:1025300003E2FC0E09C4DBFF0001F36BFC0EDB5071
:102540000001F35D1CE20001F351EA6A200FE96E1D
:10255000040EEA22EF50E66E0001F351E76EFD0E25
:10256000DBCFE9FFFE0EDBCFEAFFE750E926000EE6
:10257000EA22E552E750EF6E0001F32BDFD70401AA
:10258000180E096F400E040108170401087D880E1B
:10259000040108130001F35100D0E552E7CFD9FF41
:0225A000120027
:0E25A2006DA610D802D06DB614D80001EA055F
:1025B00009E16DBA07D0686A696A698069880001B3
:1025C000020EEA6F12006D6A696A6D860001010EE3
:1025D000EA6F12006D6A696A0001EA6B1200FADFA5
:1025E00012000001EA5101E13AD06850040B04E006
:1025F0006950040B01E038D86DB231D06850010B3E
:1026000004E06950010B01E052D86850100B04E05F
:102610006950100B01E024D86850400B04E0695069
:10262000400B01E039D86850200B04E06950200BC2
:1026300001E034D86850020B04E06950020B01E05D
:1026400034D8030E0001EA5D01E209D06850080B9E
:1026500006E06950080B03E081EC0EF0689612006A
:10266000698468986D8212006D9269946894120072
:102670000001EBA110D0F8DF6D840001080EF76FA8
:10268000070EF86F0001F707000EF85B0001F75125
:10269000F811F8E16D941200689C120070A003D04C
:1026A0000EEC10F07090689A1200689212006A6A3C
:1026B000686A9F0E6B6E7B0E696E6E6A0F0EE66E19
:1026C000710EE66E0F0EE66E14D8E552E552E55235
:1026D000160E706E68A602D06896FCD76D980EEC48
:1026E00010F00001EB910001EC6B0001030EEA6FAA
:1026F0001200D9CFE6FFE1CFD9FFFD0EDBCFE9FF16
:10270000FE0EDBCFEAFFFC0EDB5004E0EE6AFC0EAF
:0C271000DB06F9D7E552E7CFD9FF120035
:04271C0012010002A4
:1027200000000008D80401D00100010203010902E1
:102730002900010102A03209040000020300000088
:1027400009210101000122C80007058103180001C9
:102750000705010318000A0403090416034900547D
:102760000055004E0045005200200049004E004335
:102770000016034D00340020004100540058002092
:1027800000500053005500120331002E003000307D
:1027900000720065006C002E0005010980A1018512
:1027A00001098115002501750195018106950781B3
:1027B00001C00600FF0901A101150026FF00190153
:1027C00029028511750895028100190129178521B3
:1027D0009517810019012917853195178100190175
:1027E000291785329517810009018581950191008E
:1027F000090185919501910009018592950191004A
:102800000901859395019100090185949501910035
:102810001901291785989517910019012909859C97
:10282000950991001901290385A1950391001901CA
:10283000291785A2951791001901290385A39503EE
:1028400091001901291785A49517910019012902F2
:1028500085B1950291001901290285EF9502910039
:0F286000C02E272E2757275B27712787275C233A
:102870002A0EF66E000EF76E000EF86E00010900CB
:10288000F550DD6F0900F550DE6F03E1DD6701D023
:102890003DD00900F550D86F0900F550D96F0900F7
:1028A000F550DA6F09000900F550E96E0900F5509E
:1028B000EA6E090009000900F550DB6F0900F550C8
:1028C000DC6F09000900F6CFDFF0F7CFE0F0F8CFBA
:1028D000E1F0D8C0F6FFD9C0F7FFDAC0F8FF000179
:1028E000DB5302E1DC5307E00900F550EE6EDB0735
:1028F000F8E2DC07F9D7DFC0F6FFE0C0F7FFE1C080
:0E290000F8FF0001DD07000EDE5BBFD71200FE
:02290E0004D8EB
:1029100051EC0EF0FDD71200140E6F6E0001EA6B41
:102920000001EB6B0001EC6B17EC04F01200D1EC32
:0C29300012F06FBE02D0F1EC12F01200A9
:04293C0011EE00F0A8
:1029400021EE00F0F86A5F9C38EC14F0BFEC14F054
:0829500087EC14F0FBD7120024
:08295800FF0EE350E84E1200EF
:0E296000000000D000D000D0E82EFAD7120000
:02296E0000EE79
:0C29700000F00F0EEE6AEA62FDD71200C4
:02297C00030056
:02297E00120045
:10298000000000000000000000000A6400000000D9
:102990000000000000000000000000000000000037
:1029A0000000000000000000000000000000140013
:0329B00000000123
:020000040030CA
:0E0000002C8E3F1EFF8081FF6040FF600F408E
:00000001FF
